:030033000218FBB5
:0C0036009078417401F090C000E0FF22BF
:10004600E4FF74402FF582E4347BF583E0FEE5158A
:100056002404FDE43514FAA9057B01EF7C0029F997
:10006600EC3AFAEE1211F10FBF22D7E5152405F589
:1000760082E43514F583E07003020134E5152409A2
:10008600F582E43514F583E0700EE515240AF58251
:10009600E43514F583E060187F01E4FD121647E5A8
:1000A600152431F582E43514F583E054CFF0804110
:1000B600E5152406F582E43514F583E0FF1216767D
:1000C600E5152407F582E43514F583E0FF120003F5
:1000D6007F01E5152408F582E43514F583E0FD1269
:1000E6001647E5152431F582E43514F583E04430EE
:1000F600F0E5152439F582E43514F583E04480F003
:100003009078417403F090C00074BFF0907841740D
:1000130001F090C000EFF09078417403F0E51524EF
:1000230037F582E43514F583E0547F90C000F02265
:03004300021B009D
:0300000002109556
:400106009078417404F0E5152439F582E43514F583E090C000F09078417402F0E5152436F582E43514F583E0440690C000F0E515240BF582E43514F583E06032E515240C0B
:40014600F582E43514F583E0543FFFE5152437F582E43514F583EFF09078417403F0E5152437F582E43514F583E090C000F0E515240DF582E43514F583E0700302024FE588
:40018600152417F582E43514F583E06011E5152432F582E43514F583E04404F0800FE5152432F582E43514F583E054FBF0E4FFE5152432F582E43514F583E0FD121647E55E
:4001C60015240EF582E43514F583E06011E5152433F582E43514F583E04480F0800FE5152433F582E43514F583E0547FF0E5152433F582E43514F583E054FCF0E515240FEB
:40020600F582E43514F583E0602FE5152433F582E43514F583E04402F0E5152410F582E43514F583E0FF1215E7E5152411F582E43514F583E0FF121617E5152433F582E45E
:400246003514F583E0FF1215B7E5152414F582E43514F583E06044E5152415F582E43514F583E06011E5152439F582E43514F583E04401F0800FE5152439F582E43514F581
:4002860083E054FEF09078417404F0E5152439F582E43514F583E090C000F0E5152412F582E43514F583E06044E5152413F582E43514F583E06011E5152439F582E43514E6
:4002C600F583E04402F0800FE5152439F582E43514F583E054FDF09078417404F0E5152439F582E43514F583E090C000F0E5152416F582E43514F583E0FFE5152435F5820A
:40030600E43514F583EFF0E5152417F582E43514F583E030E011E5152431F582E43514F583E04440F0800FE5152431F582E43514F583E054BFF0E5152418F582E43514F576
:4003460083E0FFE515243BF582E43514F583EFF0E5152419F582E43514F583E06011E5152439F582E43514F583E04410F0800FE5152439F582E43514F583E054EFF0907869
:40038600417404F0E5152439F582E43514F583E090C000F0E515241AF582E43514F583E0606BE5152437F582E43514F583E054BFF09078417403F0E5152437F582E43514FF
:4003C600F583E0547F90C000F09078417401F0120036EF54FE90C000F0E5152432F582E43514F583E054FDFFF0FDE4FF121647E515242CF582E43514F583E4F0E515242BB7
:40040600F582E43514F583E4F0E5164213E515241BF582E43514F583E0700EE5152425F582E43514F583E06028E5152432F582E43514F583E04402FFF0FDE4FF121647E547
:4004460015242BF582E43514F5837401F0E5164213E515241CF582E43514F583E0FF700EE5152425F582E43514F583E0602A9078417402F0E5152436F582E43514F583E0C6
:40048600440490C000F0EF600FE5152431F582E43514F583E04404F0E515241DF582E43514F583E06027E5152437F582E43514F583E04440F09078417403F0E5152437F550
:4004C60082E43514F583E0547F90C000F0E515241EF582E43514F583E06028E5152432F582E43514F583E054FEFFF0FDE4FF121647E515242DF582E43514F5837401F0E58F
:40050600164213E515241FF582E43514F583E0700EE5152425F582E43514F583E06027E5152432F582E43514F583E04401FFF0FDE4FF121647E515242DF582E43514F58397
:40054600E4F0E5164213E5152420F582E43514F583E0700EE5152425F582E43514F583E060189078417402F0E5152436F582E43514F583E0440290C000F0E5152421F582A7
:40058600E43514F583E0600FE5152431F582E43514F583E04402F0E5152422F582E43514F583E0601FE515242EF582E43514F5837401F0E515243AF582E43514F583E4F0F0
:4005C600E5164213E5152423F582E43514F583E06003121885E5152424F582E43514F583E0601BE5152431F582E43514F583E04408F0907F98E0FFE516F4FEEF5EF0E5156C
:400606002425F582E43514F583E06016E5152431F582E43514F583E054F7F0907F98E04516F022907FE9E012120307830007F701086303064C0607740807680907500A07CE
:400646005F0B000008B2907FEBE024FE601C1470030206FE240260030207467419907FD4F07400907FD5F00208B9907FEAE004758217758319F0907FEAE030E0047F03802D
:40068600027F02758282758319EFF075826D758319F0758266758319F075825F758319F0758258758319F0907FEAE030E1047F6480027F3275821A758319EFF0907FEFE0FB
:4006C600FE907FEEE07C002400F519EC3EF518753319753412758214758319E0752700F528D3E5289519E527951840068518278519281213120208B9907FEAE0FF12142BC9
:40070600EA496032907FEEE0751800F519AE02AF018E338F348F828E83E0FEA3E08E27F528D39519E527951840068518278519281213120208B9907FB4E04401F00208B99E
:40074600907FB4E04401F00208B9907F00E525F0907FB57401F00208B9907FEAE0F5250208B9907FEAE0F522120AB80208B9907F00E522F0907FB57401F00208B9907FE8BD
:40078600E0247F60241460312402705BA200E433FF25E0FFA206E4334F907F00F0E4A3F0907FB57402F00208B9E4907F00F0A3F0907FB57402F00208B9907FECE0F4548063
:4007C600FFC4540FFFE054072F25E024B4F582E4347FF583E054FD907F00F0E4A3F0907FB57402F00208B9907FB4E04401F00208B9907FE8E024FE601D240260030208B910
:40080600907FEAE0B40105C2000208B9907FB4E04401F00208B9907FEAE07038907FECE0F45480FFC4540FFFE054072F25E024B4F582E4347FF583E4F0907FECE05480FF67
:40084600131313541FFFE054072F907FD7F0E04420F0805F907FB4E04401F08056907FE8E024FE60182402704A907FEAE0B40104D200803F907FB4E04401F08036907FEACB
:40088600E07020907FECE0F45480FFC4540FFFE054072F25E024B4F582E4347FF5837401F08010907FB4E04401F08007907FB4E04401F0907FB4E04402F022E511540F703D
:4008C600030209B21216A5EF20E175121703EF14F5191218CCEF2519FFE433FEC3EF9480EE648094805059851582851483E0FEA3E0FFF5828E83E030E011E5152431F58250
:40090600E43514F583E04480F0800FE5152431F582E43514F583E0547FF0E5152431F582E43514F583E020E212E519600EF523EF2401F52DE43EF52C1214ADE4FF1214E3C0
:40094600E5152431F582E43514F583E030E75D1218CCE515243BF582E43514F583E0FEEFC39E5048E515242FF582E43514F5837401F0E5152431F582E43514F583E0547B99
:40098600F0E515243AF582E43514F583E4F0E5164213907FC2E030E110E5152426F582E43514F583E0F52480031212A11216D4EF30E103020AB71217D28F191218D8E515D5
:4009C6002438F582E43514F583EFF0E5152435F582E43514F583E0FFE519C39F50281218B4EF30E021E5152438F582E43514F583E020E712E5152431F582E43514F583E0C0
:400A060020E103020AB7E5152431F582E43514F583E054FDF0E5197003020AB7B4800FE5152438F582E43514F583E04402F0E5152438F582E43514F583E0FF30E729E519CF
:400A4600D394204003751920851923851582851483A3A3E0FCA3E08C2CF52D1213DDE51925E0FF12151922E519D3943F400375193F851923E5152438F582E43514F583E053
:400A8600FF851582851483A3A3E0FCA3E0F5828C83EFF0851582851483A3A3E0FEA3E02401F52DE43EF52C12146CE51904FF12151922E4907F93F0907F9C74F0F0907F9677
:400AC600F0E4907F94F090784A04F0F58E907F9574C0F0907F9E743FF0907F98741FF090784374FFF0E4907841F0907FDF749FF0907FDEF0907F92E04402F07E7B7FC07581
:400B0600147B7515C0907F9674EFF0751601120F127E7B7FC075147B7515C0907F9674EFF0751601E5152426F582E43514F583E4F07E7E7F40851582851483747EF0A374F5
:400B460040F07E7E7F80851582851483A3A3747EF0A37480F07E7C7F0075147C751500907F9674DFF0751602120F127E7C7F0075147C751500907F9674DFF0751602E51536
:400B86002426F582E43514F5837401F07E7D7FC0851582851483747DF0A374C0F07E7E7F00851582851483A3A3747EF0A37400F07E7C7F4075147C751540907F9674BFF018
:400BC600751604120F127E7C7F4075147C751540907F9674BFF0751604E5152426F582E43514F5837402F07E7D7F40851582851483747DF0A37440F07E7D7F8085158285D3
:400C06001483A3A3747DF0A37480F07E7C7F8075147C751580907F96747FF0751608120F127E7C7F8075147C751580907F96747FF0751608E5152426F582E43514F583741C
:400C460003F07E7C7FC0851582851483747CF0A374C0F07E7D7F00851582851483A3A3747DF0A37400F0C20AC209D20222E510045403F51014601F1460311460432403701B
:400C8600527E7B7FC075147B7515C0907F9674EFF0751601803D7E7C7F0075147C751500907F9674DFF075160280287E7C7F4075147C751540907F9674BFF075160480137E
:400CC6007E7C7F8075147C751580907F96747FF0751608E53255167003020E11E516F4FF5232E526547FFE700FE52A55166024907F98E04516F0801BBE2018E5152431F543
:400D060082E43514F583E030E309E4F52A907F98E05FF0E515243AF582E43514F583E06003E014F0E5152434F582E43514F583E06003E014F0E06003020E11740AF012009D
:400D460036EF5401FFF519E515242CF582E43514F583E06F6007E519F0E51642131218E48F19E5152427F582E43514F583E0FFE5195410FE6F6006EEF0E5164213E5152415
:400D860028F582E43514F583E0FFE5195480FE6F6006EEF0E5164213E5152429F582E43514F583E0FFE5195420FE6F6015EEF0E5152431F582E43514F583E030E404E51665
:400DC6004213E5125516FFF519E515242AF582E43514F583E06F6016E519F0E5152431F582E43514F583E030E504E5164213E5175516FFF519E5152430F582E43514F58380
:400E0600E06F6007E519F0E516421322300903020F11E52414602A14604114605814606F24046003020ECF7E7B7FC075147B7515C0907F9674EFF07516011212A17524015A
:400E4600227E7C7F0075147C751500907F9674DFF07516021212A1752402227E7C7F4075147C751540907F9674BFF07516041212A1752403227E7C7F8075147C7515809051
:400E86007F96747FF07516081212A175240422300433C2045313DFE4F5197E007B00742E2519F9EE3400FA1211ABFF74802519F582E4347BF583EFF00519E519B403DB902D
:400EC6007FC37403F075240522E536603BD5360A5313EF300A04D209C20AE4F5197E007B0074352519F9EE3400FA1211ABFF74802519F582E4347BF583EFF00519E519B467
:400F060003DB907FC37403F0E4F52422E4F51A7E007B01E515251AF9EE3514FAE41211F1051AE51AB43CE8E5152435F582E43514F5837401F09078417403F0E5152437F569
:400F460082E43514F5837403F090C000F07F0CE4FD1216477F10E5152433F582E43514F583EFF01215B79078417402F07F01E5152436F582E43514F583EFF0440690C000F1
:400F8600F09078417404F0E5152439F582E43514F5837480F090C000F00FE4FD121647E4FF7EA3E5152432F582E43514F583EEF0FD1216479078417401F090C000E4F07F89
:400FC600057D7F1216477F0112154F7F037D071216472253133F907BF1E030E3167E7B7FC075147B7515C0907F9674EFF07516011208C1907C31E030E3167E7C7F00751417
:401006007C751500907F9674DFF07516021208C1907C71E030E3167E7C7F4075147C751540907F9674BFF07516041208C1907CB1E030E3167E7C7F8075147C751580907F37
:4010460096747FF07516081208C10511E511540FF518701F907841E054F7F0907F99E0F517907841E04408F0907F99E0F4F51212112122E518B40104120C7322907FC2E018
:4010860020E108E5136004120E1222120C7322787FE4F6D8FD7581370210DC021229E493A3F8E493A34003F68001F208DFF48029E493A3F85407240CC8C333C4540F44207E
:4010C600C8834004F456800146F6DFE4800B0102040810204080901850E47E019360BCA3FF543F30E509541FFEE493A360010ECF54C025E060A840B8E493A3FAE493A3F8A2
:40110600E493A3C8C582C8CAC583CAF0A3C8C582C8CAC583CADFE9DEE780BE907FD2E030E1030211AAC209907B40E014602614603B14605024836064248070637E7B7FC01C
:4011460075147B7515C0907F9674EFF0751601120046804B7E7C7F0075147C751500907F9674DFF075160212004680337E7C7F4075147C751540907F9674BFF075160412FB
:401186000046801B7E7C7F8075147C751580907F96747FF0751608120046800312175CE4907FD3F022BB010689828A83E0225002E722BBFE02E32289828A83E49322BB0189
:4011C6000CE58229F582E5833AF583E0225006E92582F8E622BBFE06E92582F8E222E58229F582E5833AF583E49322BB010689828A83F0225002F722BBFE01F322D083D086
:4012060082F8E4937012740193700DA3A393F8740193F5828883E4737402936860EFA3A3A380DF907FAEE0FFD39200E433FEEF4EF0D2E843D820907FDE7401F0907FDFF08E
:40124600907FAB74FFF0907FA9F0907FAAF05391EF907FAF7401F0907FAE740DF0D2AFD20B121814C201E4F52BF531C207C2027529F0907FD8E06526600675320FE0F526C9
:40128600300203120FD9300107C20112062980E23008DFC20812183580D822E5135516606AE515243AF582E43514F583E0705CE516F45213E5152426FFE43514FEE4FD0FA2
:4012C600EFAA0670010E14F5828A83E0FC74802DF582E4347BF583ECF00DBD0BE2907FC3740BF0E515243AF582E43514F5837410F0E515242EF582E43514F583E4F0E515C1
:40130600242FF582E43514F583E4F022E52845276057AE27AF28D3EF9440EE940040047E007F40C3E5289FF528E5279EF527E4FDEDC39FE49E501F853482853383E0FC7494
:40134600002DF582E4347FF583ECF00D0534E5347002053380DA907FA97401F0907FACE04401F0907FB5EFF022907FACE054FEF0E4907FB5F022E4907F93F0907F9C74F0A7
:40138600F0907F96F0E490784AF0907F94F0907F9D74FFF0E4907F97F0300007E52954F0FF80027F00EF4408907841F0E4907F98F0907F95F0907F9E74FFF0E4907F98F0C9
:4013C600907F93F0907F9C74F0F0E4907F96F0907F92E054FDF0228F1A052DE52DAE2C7002052C14F5828E83E51AF01218F0052DE52DAC2C7002052C14F5828C83EFF0159D
:4014060023E523601FE5152438F582E43514F583C083C082E0FE1218D88F1AEE4FD082D083F080B5228F1AE4F51B751CFF751D19751E86AB1CAA1DA91E9000011211C4B4E1
:40144600031DAF1B051BEFB51A01221211AB7E0029FFEE3AA907751CFFF51D891E80D47B007A00790022E4907841F090784F74C0F0E4907850F0E52C907851F0AE2CE52DF8
:40148600907852F0907854E523F09078577404F0907FE2E04410F0E054F7F0E4907855F0907855E060FA22E4907841F0E52C90784FF0AE2CE52D907850F090785174C0F081
:4014C600E4907852F0907854E523F09078577404F0E4907855F0907855E060FA22E5152404F582E43514F583E014600F1460131460178000907FC7EFF08013907FC9EFF081
:40150600800C907FCBEFF08005907FCDEFF0E516422A22E5152404F582E43514F583E014600F1460131460178000907FB7EFF08013907FB9EFF0800C907FBBEFF08005903B
:401546007FBDEFF0E516422A22AE07E4FFE5152432F582E43514F583E0547FFD1216479078417401F090C000EEF0E4E5152432F582E43514F583E04480FD12164722C0E0A0
:40158600C0F0C083C082C085C084C086758600C0D075D0085391EF907FA97401F0121312D0D0D086D084D085D082D083D0F0D0E0329078417403F090C00074BFF0907841D0
:4015C6007402F090C000EFF09078417403F0E5152437F582E43514F583E0547F90C000F0229078417403F090C00074BFF09078417404F090C000EFF09078417403F0E5156D
:401606002437F582E43514F583E0547F90C000F0229078417403F090C00074BFF09078417406F090C000EFF09078417403F0E5152437F582E43514F583E0547F90C000F0FF
:40164600229078417403F0E5152437F582E43514F583E0547F90C000F09078417407F090C000EFF09078417405F090C000EDF0229078417403F090C00074BFF0E4907841FA
:40168600F090C000EFF09078417403F0E5152437F582E43514F583E0547F90C000F022E5152404F582E43514F583E014600E1460111460148000907FC6E0FF22907FC8E015
:4016C600FF22907FCAE0FF22907FCCE0FF22E5152404F582E43514F583E014600E1460111460148000907FB6E0FF22907FB8E0FF22907FBAE0FF22907FBCE0FF22E515249E
:4017060004F582E43514F583E014600E1460111460148000907FC7E0FF22907FC9E0FF22907FCBE0FF22907FCDE0FF22C0E0C083C082C085C084C086758600907FC4E4F096
:401746005391EF907FAB7404F0D086D084D085D082D083D0E032907B41E0F536431310A3E06009907FD77417F07437F0907B43E0F537A3E054F0F529E06002D20A22C0E024
:40178600C083C082C085C084C086758600D2015391EF907FAB7401F0D086D084D085D082D083D0E032C0E0C083C082C085C084C086758600D2085391EF907FAB7408F0D0F7
:4017C60086D084D085D082D083D0E0321218C0AE071218C0AD07EE6D60101218C0AE07EE6D60071218C0AD0780ECAF06227400F58690FDA57C05A3E582458370F922907FD5
:40180600D6E04480F0438701000000000022907FD6E04404F0E04408F0300B04E04402F07FF47E0112186B907FD6E054F7F02212137C121804907FD6E030E70A7F057E007D
:4018460012186B12189E120AB8220335800000032E810000C185C181C108C100C106012200012400008E188F19E5191519AE18700215184E60081217F31217F380EB22E545
:40188600152404F582E43514F583E004FF4410907FD7F0EF4430F022907FD6E04401F07F0D7E0012186B907FD6E054FEF0229078417402F090C000E0FF229078417403F0D5
:4018C60090C000E0FF229078417404F090C000E0FF229078417405F090C000E0FF229078417406F090C000E0FF22E4907841F090C000E0FF2253D8EF320012011001FF00AB
:401906000040CD060A0100000102000409027400010100A032090400000EFF000000070501024000000705020240000007050302400000070504024000000705050240007A
:4019460000070506024000000705070240000007058102400001070582024000010705830240000107058402400001070585024000010705860240000107058702400001F3
:401986000403090448034B00650079007300700061006E002C002000610020006400690076006900730069006F006E0020006F006600200049006E006E006F005300790040
:4019C6007300200049006E0063002E003603550053004200200034002D0070006F00720074002000530065007200690061006C00200041006400610070007400650072003C
:401A060000000000000000000000000000000000000000000000000000000000000000000000000000000000000000000000000000000000000000000000000000000000A0
:401A46000000000000000000000000000000000000000000000000000000000000000000000000000000000000000000000000000000000000000000000000000000000060
:401A86000000000000000000000000000000000000000000000000000000000000000000000000000000000000000000000000000000000000000000000000000000000020
:401AC6000000000000000000000000000000000000000000000000000000000000000000000000000000000000000000000000000000000000000000000002178400021B26
:151B06000400021732000217AB00021B1000021B1400021584BE
:00000001FF
